:020000040000FA
:020000000C28CA
:040002000034003492
:08000800F0000308F10071088B
:080010008300F00E700E0900E0
:080018008B1383120313073060
:100020009F00831603131F308504860186178312F1
:10003000031380308605A001B101B2010130AF0089
:10004000B001822186152508AC002408AB00013ED2
:10005000AD000318250A031C2508AE00851C4128A5
:10006000A01A4628861183160313FF3092008312CC
:100070000313043092000F30970019309500A0163A
:100080004628A01E462897018615A012051D4A285D
:10009000B10F482805185428A01D53280130AF007F
:1000A000B001A001A0116428A0196328A001A01527
:1000B0002508AC002408AB00013EAD000318250A5A
:1000C000031C2508AE00A6282121201A872801300C
:1000D000AF070318B00A22082F0203182308031CD5
:1000E000230A3002031C2E28851C8528201B7F280C
:1000F0001508FF3A031D950A0319201785281508CE
:10010000193A031D95030319201320162E28AF0357
:100110002F08FF3A031D8D28B003B008031DA52842
:10012000AF08031DA528851CA428201B9E281508A0
:10013000FF3A031D950A03192017A4281508193A38
:10014000031D95030319201320122E284721201D7B
:10015000E8280130AB070318AC0AAD032D08FF3ABD
:10016000031DB328AE032D08240203182E08031C18
:100170002E0A2502031C2E28A01CD128A010013015
:10018000AB00AC012208AD002308AE00851CD028CE
:100190001508FF3A0319D028950AB20FCD28C828B0
:1001A000E72820112508AC002408AB00013EAD0073
:1001B0000318250A031C2508AE00851CE72815082E
:1001C000193A0319E7289503B20FE428DF282E28EF
:1001D0000130AD070318AE0AAB032B08FF3A031D2D
:1001E000F228AC032C08031D20292B08031D20290D
:1001F000A01C06292015851C05291508193A031984
:1002000005299503B20F0229FD28A9282508AC006D
:100210002408AB00013EAD000318250A031C250885
:10022000AE00A0181F29A014851C1E291508FF3A2E
:1002300003191E29950AB20F1B2916292029A0107F
:100240002E2886122108A900A601A7010830A800BF
:100250000130A6070318A70A0612851D0613851983
:10026000061726082F06031D3D2927083006031D03
:100270003D29851D0617851906130616A80B282982
:100280000612A90B2629861600008612080086127F
:100290002108A900A601A7010830A8000130A6077F
:1002A0000318A70A061220102B08260203182C0890
:1002B000031C2C0A2702031820142D0826020318F9
:1002C0002E08031C2E0A270203182010A0186D29DF
:1002D00020180617201C0613712920180613201C4D
:1002E0000617851D7829061B772906177829061316
:1002F0000616A80B4E290612A90B4C2986160000DB
:1003000086120800861106128612861BA017861F09
:10031000A013861B0613861F0617A201A301A101C5
:10032000A9010830A8000612000006168030060554
:10033000AA0080302005AA06031DA7290130A207C4
:100340000318A30AA80B93290612A90F91292908BB
:10035000A1002108031DB529FF30A100F830A2003B
:10036000A4000730A300A500B9292208A40023088F
:0A037000A5000310A50CA40C080062
:02400E00533F1E
:084200000000010002000300B0
:00000001FF
